:020000040000FA
:100000008501860107309F00831681130510F830A3
:1000100086008312F030F1000630F0001E30F4004C
:10002000F5011F30F9000930FA00FC01FB01051051
:100030003D300A21203084007508F600F701F801F0
:100040001130F200232805102528262827282828E3
:1000500000002A282B2800002D282E280000051437
:100060001B300A213328342800000630F000002419
:100070008000840AF60A0319F70AFF3A03190529D2
:100080000000F00B37280000F20B23288A0105102E
:1000900049284A284B284C2800004E284F280000A9
:1000A000512852280000051405300A210630F000BE
:1000B00059285A28203078078400000E860000084E
:1000C000840A6228632864280000662867280000E4
:1000D00069286A28000086006D286E2800007028B4
:1000E00071280000732874280000000EF00B5E28B1
:1000F00079287A2800007C280630F40B8028F8073D
:10010000860182281E30F4080319F400F10B4728F9
:10011000000005108B288C288D288E280000902840
:100120009128000093289428000005143B300A21F0
:1001300005109A289B289C289D2800009F28A0280D
:100140000000A228A328000005143B300A21051056
:10015000A928AA28AB28AC280000AE28AF280000A8
:10016000B128B228000005143B300A210510B82838
:10017000B928BA28BB280000BD28BE280000C02826
:10018000C1280000051434300A21F030F1000000CD
:10019000F90BCB28DC28CC28CD280000CF28D0288C
:1001A0000000D228D3280000D528D6280000D8285F
:1001B000D9280000DB281728FA0BDF28FB0A0330B8
:1001C0007B060319FB010930FA080319FA001F30F6
:1001D000F900EA2800007B088207F028F728FE28AB
:1001E0000030F50031307C18F500FC09172862302A
:1001F000F50093307C18F500FC091728C430F50091
:10020000F5307C18F500FC0917288403F603183034
:100210000A214428F3000000F30B0F2908000C29E1
:10080000043077078A000830760703188A0A8200C6
:100810000034003411341134003400340134113404
:1008200011341134113410341134113411341134A1
:1008300011341134113410340134103401341134B2
:100840001134113411341134113411340034113491
:1008500010340134113400340134103401341034B4
:1008600001341034003411340034003411340034B5
:10087000FF340034003411341134003400340134B6
:100880001134113411341134103411341134113441
:100890001134113411341134103401341034013452
:1008A0001134113411341134113411341134003431
:1008B0000134103401341034003400341134013464
:1008C0001034113400341134003400340034003456
:1008D0001134FF3400342034003400342034003428
:1008E0000034023400340234003400340034223442
:1008F0002234223420340034023420342234203490
:10090000223400342234223422342234223420345B
:100910002034223422342234203420342034203431
:1009200000340034203420340034023420342234A3
:1009300000340034FF3400342034003400342034D8
:1009400000342034023400340234003420342034A3
:1009500022342234223420342034223420342234ED
:1009600020342234203422342234223422342234DB
:10097000203402342234223422342034003400342F
:100980002034003400342034003402340034003485
:10099000003402340034FF34003400340434403472
:1009A000003400340034003444344434003400341F
:1009B0000034043444344434403400340034443487
:1009C0000434403444340034003444344434443433
:1009D00044340034003400344034043400340034EF
:1009E000003404340434403440340034003440349F
:1009F0004034043404340034FF340034003404340C
:100A0000403400340034003400344434443400347E
:100A1000003400340434443444344034003400346A
:100A200044340434403444340034003444344434D2
:100A30004434443400340034043404344034403406
:100A400000340034403400340034043400340034C2
:0C0A500004340034003440340034FF341F
:02400E00623F0F
:00000001FF
